:020000040000FA
:100000000129FF3FFF3F8312031321088A002008C4
:1000100082000800831203137008F100F001083019
:10002000FC007108F40C03181928FC0B1228F101CC
:10003000003403101E28F40C0318F107F10CF00C27
:10004000FC0B1B28080083120313FB01FA01F901C2
:100050008030F800F10CF00C031C37287408F90705
:1000600075080318750FFA070318FB0A0310F01F31
:100070003F287408FA0775080318750FFB07FB0C77
:10008000FA0CF90CF80C031C2A287B08F3007A08F8
:10009000F2007908F1007808F000080010308312AF
:1000A0000313860010100C11221008008312031392
:1000B000A901AA01051E5E282030A907851F622814
:1000C0001030A907851D66280830A907051C6A2875
:1000D0000430A907051D6E280230A907851C712868
:1000E000A90A061D75280430AA00861C792802304A
:1000F000AA07051F7C28AA0AD0282908A700A8015A
:10010000F0282908F0000530F4000A207008A70044
:100110007108A800F0282908F0000F30F4000A2028
:100120007008A7007108A800F0282908F0003C30EA
:10013000F4000A207008A7007108A800F028290818
:10014000F0007830F4000A207008A7007108A800B9
:10015000F0282908F000F1012C30F4000130F500FE
:1001600023207008A7007108A800F0282908F000D3
:10017000F1015830F4000230F50023207008A70088
:100180007108A800F0282908F000F1018430F4007B
:100190000330F50023207008A7007108A800F0289C
:1001A0002A08003A03197D282A08013A03198128F0
:1001B0002A08023A03198B282A08033A03199528BA
:1001C0002A08043A03199F282A08053A0319A9287E
:1001D0002A08063A0319B6282A08073A0319C32839
:1001E0002708F0002808F100080003208A110A12ED
:1001F0008000840AA00A0319A10AF003031DF52850
:1002000008000730831203139F0010308600850119
:10021000CF3083168600FF308500011383128E01D4
:100220008F0110129012901490150B309700FF3030
:1002300095003F3096000C118B102210A210562012
:100240007008A5007108A6000C1D3E290C11103085
:100250008606A21C372901302302F0000030031C5F
:10026000013E2402F1007008A3007108A4002308D5
:100270002404031D3C294E200230A206851A412980
:100280004E208B1C6C298B10851E6C2922185B2933
:100290008F010F088E0010140C11203086002214DC
:1002A000A21056207008A5007108A6002508A3001A
:1002B0002608A4006C29861D6C298F010F088E006A
:1002C00010140C11A21056207008A5007108A60089
:1002D0002508A3002608A40024296D29FF3FFF3F1D
:1002E000FF3FFF3FFF3FFF3FFF3FFF3FFF3FFF3F1E
:1002F000FF3FFF3FFF3FFF3FFF3FFF3FFF3FFF3F0E
:10030000FF3FFF3FFF3FFF3FFF3FFF3FFF3FFF3FFD
:10031000FF3FFF3FFF3FFF3FFF3FFF3FFF3FFF3FED
:02400E00503F21
:08400000FF3FFF3FFF3FFF3FC0
:00000001FF
